:1078000011E0A0E0B1E0E6EDFFE702C005900D92C7
:10781000A630B107D9F721E0A6E0B1E001C01D9282
:10782000AD34B207E1F7CDB7DEB72897DEBFCDBFE5
:10783000112484B78093270114BE88E180936000EF
:1078400089E280936000259A86E020E295B1922734
:1078500095B93FE748E391E0315040409040E1F76F
:1078600000C00000815091F78091270181FF72C014
:1078700082E08093C00088E18093C10086E080931D
:10788000C20080E18093C40010E000E0D12CC12C44
:10789000AA24AA94BA2C99249394A895F6D1813459
:1078A00071F4F3D1F82E3FD3E2E8FE1202C083E078
:1078B00004C0F1E885E6FF12FACF2ED304C082346B
:1078C00021F484E13CD3F12C40C0853411F485E0EF
:1078D000F9CF853541F4D9D1082FD7D1182F000F12
:1078E000111F21D3F0CF863521F484E028D380E026
:1078F000E4CF8436D9F4C9D1C8D1882EC6D1C80CFA
:10790000D11CF12CF81418F0C801CBD1EACFBDD1AD
:10791000E82EBBD1F801EF0DF11D982F8E2D0C0133
:1079200097BEE8951124F394F394ECCF843709F0D3
:107930008BC0ABD1AAD1F82EA8D1F5D2F801859190
:107940008F01EAD2FA94F110F9CF80E1E5D2FF205D
:1079500009F4A3CF8EE284B981E58CBD81E08DBDB1
:10796000512C412C77247394AA24AA94BA2C8824ED
:10797000839473E0972EEAE06E2EF999FECF43E0F0
:1079800050E070E060E089E291E003D348E050E02D
:107990006BE171E0CE010196FCD229982A9A63E04E
:1079A00083E2EBD166E685E2E8D167E286E2E5D1E3
:1079B00063E780E5E2D164E08DE3DFD161E082E25C
:1079C000DCD161E081E2D9D161E08CE3D6D121E064
:1079D00041E070E060E086E0A3D18732F9F4809165
:1079E0002A01809328018FEF80932A0180932B0135
:1079F0008093080163E584E2C0D143E26AE087E056
:107A000083D161E08EEFD8D1109208016FE584E256
:107A1000B4D180912A018F3F09F0A0C08D819E8151
:107A200024E0880F991F2A95E1F74DD12F813885E1
:107A30008217930709F0A1CF1CBCA895809127015C
:107A4000282EF201099599CF853739F46CD28EE151
:107A500063D285E961D28FE030CF813509F041CF23
:107A6000BA82A982BC82AB82C601F4E09695879562
:107A7000FA95E1F79E838D83C60125D198878F8380
:107A8000CE01019663D24FD2FF24F3945ECF8701DB
:107A900089819A8190930E0180930D018B819C8145
:107AA0009093100180930F01780181E0E81AF108AA
:107AB000F0921201E092110144EC62E382E024D1E1
:107AC00063E083E079D1882309F46BC046E050E09D
:107AD00063E371E08DE091E04FD2892BC9F6C801D4
:107AE0008150904F682F62956077ACE2B1E0462FED
:107AF00050E04C525140FA01EA0FFB1F1E963C9198
:107B00001E971D962C911D97090177BEE8951124AB
:107B10001296E1E0AC33BE0771F7611106C044E094
:107B2000880F991F4A95E1F7BCD0E114F10409F0E0
:107B3000AECFD886CF828D819E8134E0880F991F89
:107B40003A95E1F7C0D0C816D90621F01E821D82F1
:107B500018861F82CE010196F9D10FCF809129019D
:107B600081508E3FF0F043E262E083E0CDD063E0ED
:107B700084E022D1882391F380912F018695869508
:107B80008695E3E3F1E060E0815020F490E080E04E
:107B900010D2F3CE9191669D900D1124692F605300
:107BA000F3CF70920D0110920E0143EC62E18FE071
:107BB000ABD060E08FE000D18D819E8154E0880FD2
:107BC000991F5A95E1F77FD098878F8388E0FE014F
:107BD0003196ADE0B1E001900D928A95E1F7909277
:107BE00016018092150144EC62E580E08DD063E0DF
:107BF00081E0E2D0882309F411CF48E050E063E34C
:107C000071E0CE010196B8D1892B09F407CF00911C
:107C10003701109138010115110501F580913901E5
:107C200090913A018A379A4DE9F48091330190910D
:107C300034018130910551F46FEFC801BAD10F5F63
:107C40001F4F011534E01307B9F797CE0297823022
:107C5000910508F092CE609135019ACF0038174017
:107C600008F0DCCE88E0E3E3F1E0DE01119601905C
:107C70000D928A95E1F7CF80D884B886AF82CE0185
:107C8000019664D10D811E8103CF8091C00087FFD2
:107C9000FCCF8091C00084FD01C0A8958091C600F2
:107CA000089523E0FC0127BFE89507B600FCFDCF4F
:107CB00025E0FC0127BFE89507B600FCFDCF81E178
:107CC00087BFE8950895BC01F0E0E0E08FEF9FEFFB
:107CD000E617F70720F4E11528E7F20708F0089502
:107CE0002591822748E0DC01B695A79581709927F8
:107CF00022273327281B390B2170307ACD018227A8
:107D00009327415081F7E4CF90912901E6E0F1E01B
:107D1000918390839FEF9683858344836383089543
:107D20002A989AE19A95F1F700C08EBD0DB407FE2E
:107D3000FDCF8EB59FEF415030F42A9ABAE1BA9543
:107D4000F1F700C00895222369F09EBD0DB407FE2F
:107D5000FDCF8EB56115710571F3DB018C936F5FFB
:107D60007F4FE9CFFB013196DB018C918EBD0DB4C5
:107D700007FEFDCF8EB5BF01DECFCF93DF931F92FD
:107D8000CDB7DEB7698320E041E0BE016F5F7F4F72
:107D9000C7DF0F90DF91CF91089520E040E070E0C1
:107DA00060E082EEBDDF20E040E070E060E081EE68
:107DB000B7DF60E787E2E1CFFF920F931F93CF9386
:107DC000DF93C82FF62ED0910901D695D695D6957A
:107DD000D95F10912A0129986EE080E2CEDF1093DE
:107DE000000120E045E060E071E08AE299DF20E0F8
:107DF00045E060E071E080E393DF20E04D2F66E036
:107E000071E080EA8DDF299A8AE08A95F1F700C057
:107E100020E040E070E060E08FEF82DF8073C1F32C
:107E20002998BBDF6FE080E2A8DF609129018AE238
:107E3000A4DF299A0FEF1FEFA89521E041E070E041
:107E400060E087E16DDF80FF1AC09FEF88E08A95D0
:107E5000F1F70150110919F0C913EECF9C2FFA94D4
:107E60008FEFF81619F0C913AECF9C2F81E0C9131C
:107E700080E0DF91CF911F910F91FF90089521E055
:107E800041E070E060E080E64BDFD82F813208F0FF
:107E9000D0E021E04D2F6CE271E081E641DF7DDF33
:107EA00080912F0186958695869590E00796D81744
:107EB000190659F690912E01809129019813C5CF8A
:107EC00090913101809130018770833009F0BECFED
:107ED000983009F0BBCF8091280120912A01281306
:107EE00003C08F3F09F0B2CF20912D01821304C04F
:107EF00080932A019EEFAACF3091330181E0830F56
:107F00008093330140912B01341708F09FCF809369
:107F10002B0120932A019ACF9091C00095FFFCCFAE
:107F20008093C6000895B1DE803239F088E18093F5
:107F3000600088E080936000FFCF84E1EDCFCF93B5
:107F4000C82FA3DEC150E9F7CF91EDCF0F931F9358
:107F5000CF93DF938C01CBE1D1E0F80161918F01E8
:107F6000CE0127D02196C332F1E0DF07B1F7DF91D0
:107F7000CF911F910F910895FB01DC0104C08D91F9
:107F80000190801921F441505040C8F7881B990B8B
:107F90000895DC01CB01FC01F999FECF06C0F2BDCA
:107FA000E1BDF89A319600B40D9241505040B8F7B7
:107FB0000895262FF999FECF92BD81BDF89A0197B9
:107FC00000B4021639F01FBA20BD0FB6F894FA9A21
:067FD000F99A0FBE0895AE
:067FD60000FCE1A8A80078
:107FDC00040000001400000003000000474E550090
:107FEC00BD84295F154499570D31AA9FD5E04F46A2
:047FFC003C997B60D1
:040000030000780081
:00000001FF
